:1000000050C0BBC167C066C065C064C063C062C089
:1000100061C060C05FC05EC05DC05CC05BC05AC0F4
:1000200059C058C057C009022200010100800A09C6
:100030000400000103000000092101010001221653
:100040000007058103080064120110010000000888
:10005000C016DF05000101020001140341006E001B
:1000600061006C00470061007500670065001A03BD
:100070006E0065006F002D0073006F006600740055
:100080002E006F0072006700040309040600FF09D8
:1000900001A101150026FF00750895800900B20234
:1000A00001C011241FBECFEDCDBF10E0A0E6B0E02F
:1000B000E8E6F6E002C005900D92A236B107D9F746
:1000C00020E0A2E6B0E001C01D92AF38B207E1F730
:1000D000A7D2C8C295CFCF93DF93609175006350CC
:1000E00067FDBEC080917200CCE0D0E0C81BD10992
:1000F000C758DF4F809171008D3209F0A0C0683081
:1001000009F0ACC083EC809365008AE580936100C0
:10011000109262008881807631F0CE0170D28F3FDC
:1001200009F47CC082C08A8110926E00998191117D
:1001300006C010926F002EE630E082E06AC0953073
:1001400019F48093760057C0963009F04EC09B8119
:10015000913041F488E490E09093740080937300B0
:1001600082E13FC0923041F486E290E090937400C7
:100170008093730082E235C09330F1F4811108C09E
:1001800088E890E0909374008093730084E029C025
:10019000813041F48EE690E0909374008093730078
:1001A0008AE11FC08230E1F48AE590E09093740008
:1001B0008093730084E115C0913241F488E390E0AC
:1001C000909374008093730089E00BC0923241F4E5
:1001D0008CE890E0909374008093730086E101C0F6
:1001E00080E090E49093620020C0983079F09930DC
:1001F00031F4809378002EE630E080E00AC081E0A0
:100200009A3009F080E02EE630E003C028E730E0C5
:1002100081E0309374002093730007C0988197FDAC
:100220008E8190E89093620007C09F81911104C075
:100230009E81981708F4892F809360000FC08091E9
:10024000620087FF0BC0CE01BFD18F3F21F48EE14A
:100250008093610003C081111092600010927500BC
:100260008091610084FF5CC0809160008F3F09F441
:1002700057C0C82F893008F0C8E08C1B80936000FD
:100280008091650098E8892780936500CC23B9F1B7
:100290008091620087FF08C06C2F86E690E085D1D0
:1002A000C82F8930B8F52BC02091730030917400AD
:1002B00086FF12C0A6E6B0E045E650E040955095B6
:1002C000420F531F8C2F8A0FFA01EA0FFB1FE49194
:1002D000ED938A13F9CF09C0E6E6F0E0D9018C2F3F
:1002E0008E0F9D9191938E13FCCF2F5F3F4F8FEF19
:1002F0008C0F280F311D30937400209373006C2FE6
:1003000086E690E036D0CC5FCC3041F08FEF809322
:10031000600004C08FEF80936000CEE1C093610065
:1003200084E190B3947131F48150D9F71092760042
:1003300010927000DF91CF91089585B7826085BFDC
:100340008BB780648BBF0895A82FB92F80E090E011
:1003500041E050EA609530E009C02D9182279795E1
:10036000879510F084279527305EC8F36F5FA8F358
:100370000895EADF8D939D930895CF93CFB7CF93E0
:10038000DF93C395849BE9F7849B0BC0849B09C0D2
:10039000849B07C0849B05C0849B03C0849B01C0D1
:1003A0008BC06F93C0917200DD27C758DF4F2F932A
:1003B00065E5849B03C02F916F91E6CF0F931F9348
:1003C0004F9320E040E15F9300B3047104FB27F9F1
:1003D0003F9350E03BE039C0147140642F77012F08
:1003E0005F5F1EC0406810B314712F7752501FC05A
:1003F000406400B32F770471D1F15F5F00C023C068
:10040000406210B32F77147191F15F5F00C025C077
:1004100004711027515012F45D5F000011502795B0
:100420002C3F10B3C8F614710127015027952C3FBB
:10043000C8F64227499300B3047110274F73115037
:1004400027952C3FA8F64695469510B3147179F080
:100450000127015027952C3F98F66B5A60F33150D5
:1004600000B3B0F600C010E41ABF002719C03B501B
:100470003195C31BD04010E41ABF0881033C09F139
:100480000B34F9F0209170001981110F1213EDCF88
:100490004A81441F093651F10D3211F0013E29F70E
:1004A000009377003F915F914F911F910F912F9192
:1004B0006F91CAB7C6FD65CFDF91CF91CFBFCF9106
:1004C000189520917700222369F31091750011236C
:1004D00049F534304AF13093750020937100109142
:1004E00072003BE0311B309372001EC0009175001A
:1004F0000130C4F40AE54F70A9F43091610034FD75
:1005000014C000936100C5E6D0E013C0052710E0D9
:1005100000C0000002BB1AC0052710E0221F1DC04A
:1005200010E021C04AE502C032ED432FC4E1D0E023
:1005300032E011B31461949A02B311BB54E120E884
:1005400065E320FF052702BB279517951C3FF0F6B2
:100550006695B8F7B1F720FF052702BB27951795D9
:100560001C3FD0F62795179517FF052700001C3F65
:1005700002BBB0F629913A9519F70B7E10917600DF
:10058000110FC651D04002BB11F01093700010E45F
:100590001ABF006111B31B7E402F4B7E54E05A9569
:1005A000F1F702BB11BB42BB7DCF90916300862F58
:1005B000961708F4892F20916400280F2093640077
:1005C000981B909363000895209163002223A9F063
:1005D000261708F4622FFC01808186BF8091640099
:1005E000860F8093640090916300961B9093630044
:1005F00081E0992319F080E0089581E00895FC01DD
:1006000020812076203251F48181893039F481E0D3
:1006100080936300109264008FEF089580E0089546
:100620002EE088E190E00FB6F894A89581BD0FBE4A
:1006300021BD83DE8C9A80E0815041F0A895EFE9DE
:10064000FFE03197F1F700C00000F6CF8C98BA9A1E
:1006500081E880BF80E186BF82E083BF7894A8955F
:080660003ADDFDCFF894FFCF55
:02066800FF5A37
:00000001FF
